:020000001028C6
:10000800FE00030EF1000408F2000A08F300831250
:1000180003137F08F400562897288B0107308312B2
:1000280003139F0001308316031385008312031303
:1000380085010230831603138600023083120313EE
:100048008600063081008B16043083160313810066
:100058007D30F5007508F900F801F601F701831203
:100068000313061083208B17831203130616051833
:100078003F288616402886128C1E3B280430F5003F
:100088007508F6008C1298184B28181D5128981CD2
:100098004F2818121816181D3B281A08F50075085D
:1000A800F7003B280B1D78280B1106308100013022
:1000B800F902F908031D68287D30F0007008F9007E
:1000C8000430F0007008F800780803196F28013030
:1000D800F8028615702886117608031977280130EA
:1000E800F6028514782885107408FF0073088A00C2
:1000F80072088400710E8300FE0E7E0E09008316BE
:10010800031318150C30990018128312031398174B
:100118001813831603131813831203131816831660
:10012800031398160800F601F701F8018301112856
:02400E0061FF50
:00000001FF
